:1000000033C10000A8C600007BC600004EC6000039
:1000100021C60000F4C50000C7C5000055C100009E
:1000200053C1000051C100004FC100004DC100008C
:100030004BC1000049C1000047C1000045C100009C
:1000400043C1000041C100003FC100003DC10000AC
:100050003BC1000039C1000037C100005BC5000092
:1000600033C1000021C50000F6C400002DC100000E
:100070002BC1000029C1000027C1000025C10000DC
:1000800023C1000021C100001FC100001DC10000EC
:100090001BC1000019C1000017C1000015C10000FC
:1000A00013C1000011C100000FC100000DC100000C
:1000B0000BC1000009C1000007C1000005C100001C
:1000C00003C1000001C10000FFC00000FDC000002E
:1000D000FBC00000F9C00000F7C00000F5C0000040
:1000E000F3C000002F0A002300230023005C232319
:1000F00023235265616C53696D476561722300006B
:100100000020002300260029002C002F00320000D0
:1001100001000003010601090100000A0B02090C9D
:100120000D0E08070304010000000000000000009D
:1001300000000000000000000000000000000000BF
:10014000000000000012111000000000000000007C
:10015000000000000000000000000000000000009F
:10016000002200250028002B002E00310034000260
:10017000010000050108010B0100002100240027F7
:10018000002A002D003000330001010000040107A7
:10019000010A01050505050705080808080202020D
:1001A000020A0A0808040404040101010101010112
:1001B000010303030303030303040707070C0C0CE9
:1001C0000C0C0C0C0C0202020206060606060606C1
:1001D000060B0B0B0B0B0B0B0B010210202008085E
:1001E0001020401020408002010201080402010199
:1001F0000204081020408080402010080402018082
:1002000004020180402010080402010804020101D8
:100210000204081020408001020408102040802FB2
:100220000A002300230023005C232323235265615B
:100230006C53696D4765617223000A003D300A0006
:100240003D310A000A000A002F0A00230023002380
:10025000005C232323235265616C53696D476561FC
:10026000722300007207690B11241FBECFEFD1E289
:10027000DEBFCDBF00E00CBF26E0A4EEB3E001C0BE
:100280001D92AB31B207E1F713E0A0E0B2E0EAE083
:10029000FCE100E00BBF02C007900D92A43EB10745
:1002A000D9F711E0C3E3D1E000E006C021970109CE
:1002B000802FFE010E94D30BC233D10780E00807D4
:1002C000A9F7D6D60C94F40D9BCEAF92BF92CF92E5
:1002D000DF92EF92FF920F931F93CF93DF936C0106
:1002E0007B018B01040F151FEB015E01AE18BF08E7
:1002F000C017D10759F06991D601ED91FC91019099
:10030000F081E02DC6011995892B79F7C501DF91A0
:10031000CF911F910F91FF90EF90DF90CF90BF9002
:10032000AF900895E1EBF4E04481558160817181E3
:100330008BE094E0CACFFC01538D448D252F30E033
:10034000842F90E0821B930B541710F0CF960895E2
:1003500001970895FC01918D828D981761F0A28D0F
:10036000AE0FBF2FB11D5D968C91928D9F5F9F73D5
:10037000928F90E008958FEF9FEF0895FC01918D8B
:10038000828D981731F0828DE80FF11D858D90E0F8
:1003900008958FEF9FEF0895FC01918D228D892F95
:1003A00090E0805C9F4F821B91098F73992708957D
:1003B0008BE094E0F1DF21E0892B09F420E0822F2B
:1003C0000895FC01A48DA80FB92FB11DA35ABF4FEA
:1003D0002C91848D90E001968F739927848FA68944
:1003E000B7892C93A089B1898C91837080648C9398
:1003F000938D848D981306C00288F389E02D808147
:100400008F7D80830895EF92FF920F931F93CF9378
:10041000DF93EC0181E0888F9B8D8C8D98131AC03F
:10042000E889F989808185FF15C09FB7F894EE8926
:10043000FF896083E889F989808183708064808383
:100440009FBF81E090E0DF91CF911F910F91FF90CE
:10045000EF900895F62E0B8D10E00F5F1F4F0F7376
:100460001127E02E8C8D8E110BC00FB607FCFACF32
:10047000E889F989808185FFF5CFCE01A2DFF2CF2F
:10048000EB8DEC0FFD2FF11DE35AFF4FF0829FB76C
:10049000F8940B8FEA89FB8980818062D0CF0F931B
:1004A0001F93CF93DF938C01D0E0C0E0F801EC0FF5
:1004B000FD1F6491662339F08BE094E0A4DF892B63
:1004C00011F02196F3CFCE01DF91CF911F910F91C3
:1004D0000895CF93DF93EC01888D8823B1F0AA892A
:1004E000BB89E889F9898C9185FD03C0808186FDEF
:1004F0000CC00FB607FCF7CF8C9185FFF2CF80813F
:1005000085FFEDCFCE015DDFEACFDF91CF9108957A
:10051000CF93DF9390E0FC01E752FE4F24918D567C
:100520009E4FFC0184918823C9F090E0880F991FA9
:10053000FC01E758FE4FA591B491FC01E15AFE4F32
:10054000C591D49161110DC09FB7F8948C912095FD
:1005500082238C938881282328839FBFDF91CF91AA
:100560000895623051F49FB7F8943C91822F8095A2
:1005700083238C93E8812E2BEFCF8FB7F894EC91E7
:100580002E2B2C938FBFEACF3FB7F8948091F703BF
:100590009091F803A091F903B091FA0326B5A89BB6
:1005A00005C02F3F19F00196A11DB11D3FBFBA2F05
:1005B000A92F982F8827BC01CD01620F711D811DC5
:1005C000911D42E0660F771F881F991F4A95D1F74A
:1005D00008958F929F92AF92BF92CF92DF92EF9247
:1005E000FF924B015C01D0DF6B017C01CDDF6C1908
:1005F0007D098E099F09683E734081059105B0F31E
:1006000021E0821A9108A108B10888EEC80E83E0A3
:10061000D81EE11CF11C81149104A104B10431F72E
:10062000FF90EF90DF90CF90BF90AF909F908F9012
:1006300008952FB7F8946091F3037091F4038091BB
:10064000F5039091F6032FBF0895862F642F60CF96
:10065000FC01218530E0F901E75EFE4F8491F9014C
:10066000E752FE4F94912D563E4FF90124912223DB
:1006700009F430C0882311F181508231F8F4E82F59
:10068000F0E08827E95BFC4F8F4F0C94D30B750388
:10069000790359036D0371035E037C0382038603B0
:1006A0008C03900394039A039E035E03A203A803A2
:1006B000AC03809180008F7780938000E22FF0E080
:1006C000EE0FFF1FE150FF4FA591B491EC919E23D7
:1006D00081E009F480E081700895809180008F7D31
:1006E000EBCF80918000877FE7CF84B58F7784BD83
:1006F000E5CF84B58F7DFBCF8091B0008F7780935D
:10070000B000DCCF8091B0008F7DF9CF8091900058
:100710008F7780939000D2CF809190008F7DF9CF1A
:1007200080919000877FF5CF8091A0008F77809394
:10073000A000C4CF8091A0008F7DF9CF8091A00050
:10074000877FF5CF809120018F7780932001B6CFEE
:10075000809120018F7DF9CF80912001877FF5CF97
:10076000DC01ED91FD918081ED91FD919081ED9104
:10077000FD916C9163708E2309F064609F2309F0F2
:100780006860EDECF3E0E60FF11D659565956D93FE
:100790006D917D918D919D91099423C01AC012C0D5
:1007A00016C010C01EC009C014C013C006C019C0B6
:1007B00009C00DC007C00DC014C062507040804019
:1007C00090400BC0615070408040904006C06E5F0A
:1007D00001C06F5F7F4F8F4F9F4F9E938E937E938D
:1007E0006E930895CF93DF93EC018B85823058F49C
:1007F000F894CE01B5DF6F81788589859A857894E4
:10080000DF91CF910895F894F6CF8F929F92AF9297
:10081000BF920F931F93CF93DF93CDB7DEB7A1970E
:100820000FB6F894DEBF0FBECDBF19A2423008F458
:100830004AE08E010F5D1F4F842E912CB12CA12C0C
:10084000A501940172D7E62FB901CA01EA303CF53F
:10085000E05DD801EE938D01232B242B252B81F70E
:1008600090E080E0109761F0FD0101900020E9F731
:100870003197AF014A1B5B0BBD018BE094E025DD96
:10088000A1960FB6F894DEBF0FBECDBFDF91CF911A
:100890001F910F91BF90AF909F908F900895E95C4A
:1008A000D8CF4AE061E070E080E090E0AECF009702
:1008B00061F0FC0101900020E9F73197AF01481B7E
:1008C000590BBC018BE094E000CD90E080E00895EE
:1008D0008BE094E061DD892B99F18BE094E03ADDC7
:1008E0008C37C1F48DEE90E0DADD8EE692E0DFDF4A
:1008F0008BEE90E0D4DDD5DF89EE90E0D0DD84E0B2
:1009000092E0D5DF87EE90E0CADD0CDD84EE90E06A
:10091000C6DDDECF8C3329F41092F1031092F00380
:10092000D7CF8A30C9F38091F0039091F1038436D8
:10093000910594F701969093F1038093F003C8CF4B
:10094000089536DD8111C4DF80E090E0892B49F005
:1009500080E090E0892B29F00E94000081110E9424
:10096000000080E090E0892B49F080E090E0892B46
:1009700029F00E94000081110E94000080E090E0B8
:10098000892B49F080E090E0892B29F00E9400003B
:1009900081110C9400000895CF93DF93EC018881BE
:1009A0009981009709F0A3D7198218821D821C82B1
:1009B0001B821A82DF91CF910895FC018081918181
:1009C000009709F094C708950F931F93CF93DF9377
:1009D000EC0188819981009759F02A813B81261783
:1009E000370730F081E0DF91CF911F910F9108958B
:1009F0008B016F5F7F4F0E94000D009759F0998324
:100A000088831B830A832C813D81232B59F7FC01AA
:100A10001082E8CF80E0E7CFEF92FF920F931F9311
:100A2000CF93DF93EC017B018A01BA01CDDF811105
:100A30000AC0CE01B1DFCE01DF91CF911F910F919E
:100A4000FF90EF9008951D830C83B70188819981F1
:100A50000E94ED0DF0CF1F920F920FB60F9211244E
:100A60000BB60F922F933F934F935F936F937F93A8
:100A70008F939F93AF93BF93EF93FF938BE094E09B
:100A8000A0DCFF91EF91BF91AF919F918F917F91EA
:100A90006F915F914F913F912F910F900BBE0F90EF
:100AA0000FBE0F901F9018951F920F920FB60F92C6
:100AB00011240BB60F922F938F939F93EF93FF9375
:100AC000E0911B04F0911C048081E0912104F091DD
:100AD000220482FD1DC09081809124048F5F8F735A
:100AE00020912504821741F0E0912404F0E0E55FB5
:100AF000FB4F958F80932404FF91EF919F918F91ED
:100B00002F910F900BBE0F900FBE0F901F90189556
:100B10008081F2CF1F920F920FB60F9211242F9364
:100B20003F938F939F93AF93BF938091F3039091E3
:100B3000F403A091F503B091F6033091F20323E0A2
:100B4000230F2D3758F50196A11DB11D2093F203F7
:100B50008093F3039093F403A093F503B093F6030B
:100B60008091F7039091F803A091F903B091FA03F3
:100B70000196A11DB11D8093F7039093F803A093F4
:100B8000F903B093FA03BF91AF919F918F913F9179
:100B90002F910F900FBE0F901F90189526E8230FEE
:100BA0000296A11DB11DD2CF1F920F920FB60F92C8
:100BB00011240BB60F922F933F934F935F936F9334
:100BC0007F938F939F93AF93BF93EF93FF93809106
:100BD000E6039091E703C4DDFF91EF91BF91AF91E0
:100BE0009F918F917F916F915F914F913F912F9145
:100BF0000F900BBE0F900FBE0F901F9018951F9275
:100C00000F920FB60F9211240BB60F922F933F93B2
:100C10004F935F936F937F938F939F93AF93BF9304
:100C2000EF93FF938091E4039091E50399DDFF91A9
:100C3000EF91BF91AF919F918F917F916F915F9154
:100C40004F913F912F910F900BBE0F900FBE0F90C1
:100C50001F9018951F920F920FB60F9211240BB68A
:100C60000F922F933F934F935F936F937F938F9345
:100C70009F93AF93BF93EF93FF938091EE03909177
:100C8000EF036EDDFF91EF91BF91AF919F918F9137
:100C90007F916F915F914F913F912F910F900BBE7C
:100CA0000F900FBE0F901F9018951F920F920FB6C6
:100CB0000F9211240BB60F922F933F934F935F9394
:100CC0006F937F938F939F93AF93BF93EF93FF9314
:100CD0008091EC039091ED0343DDFF91EF91BF9183
:100CE000AF919F918F917F916F915F914F913F91C4
:100CF0002F910F900BBE0F900FBE0F901F90189565
:100D00001F920F920FB60F9211240BB60F922F93D2
:100D10003F934F935F936F937F938F939F93AF9383
:100D2000BF93EF93FF938091EA039091EB0318DD5B
:100D3000FF91EF91BF91AF919F918F917F916F91B3
:100D40005F914F913F912F910F900BBE0F900FBE6F
:100D50000F901F9018951F920F920FB60F921124AB
:100D60000BB60F922F933F934F935F936F937F93A5
:100D70008F939F93AF93BF93EF93FF938091E8037B
:100D80009091E903EDDCFF91EF91BF91AF919F91BD
:100D90008F917F916F915F914F913F912F910F9024
:100DA0000BBE0F900FBE0F901F90189590E08230F1
:100DB00090F404968330910569F17CF481309105BB
:100DC000C9F00297F9F0809169008C7F816080936F
:100DD0006900E89A08950297EDCF8430910511F1EA
:100DE000059789F780916A00837F846080936A0009
:100DF000ED9A089580916900837F846080936900F3
:100E0000E99A0895809169008F7C806180936900E0
:100E1000EA9A0895809169008F73806480936900D5
:100E2000EB9A089580916A008C7F816080936A00BC
:100E3000EC9A089580E008950F931F93CF93DF936A
:100E4000EC01062F142F62E0802F62DB62E0812F1D
:100E50005FDB802F90E0FC01ED56FE4FE491F0E067
:100E6000EE0FFF1FE150FF4FA591B491B983A88306
:100E7000FC01E752FE4F24912C83812F90E0FC016E
:100E8000ED56FE4FE491F0E0EE0FFF1FE150FF4FF3
:100E9000459154915B834A83FC01E752FE4FE491F4
:100EA000ED831F82188619861A868BE39FE10197CE
:100EB000F1F78C91282391E009F490E0DA018C910C
:100EC000E82309F092609E83BE01802FB3DF082FD4
:100ED000BE01812FAFDF800F8B87DF91CF911F91F4
:100EE0000F91089510920E0410920D0488EE93E075
:100EF000A0E0B0E080930F0490931004A09311043D
:100F0000B093120488E592E090930C0480930B0454
:100F100085EC90E0909318048093170484EC90E0A3
:100F200090931A048093190480EC90E090931C0431
:100F300080931B0481EC90E090931E0480931D0429
:100F400082EC90E09093200480931F0486EC90E064
:100F5000909322048093210410922404109225047B
:100F60001092260410922704A8EAB4E090E080E0F2
:100F700041E2FC013E9621E030E08630910510F41C
:100F800030E020E0E20FF31F40935700E491ED932F
:100F900001968930910569F74EE16FE187ED95E0A3
:100FA0004BDF81E892E09093E4058093E30582E9CA
:100FB00092E09093E6058093E5054EE26FE287EEBE
:100FC00095E03ADF83EA92E09093F4058093F3058D
:100FD00084EB92E09093F6058093F50545E364E396
:100FE00087EF95E029DF85EC92E0909304068093EB
:100FF000030686ED92E0909306068093050643E390
:1010000062E387E096E018DF87EE92E090931406A3
:101010008093130688EF92E090931606809315064E
:10102000E7EBF4E02AE632E08AE090E031832083C7
:10103000128213821482158297838683108611860A
:10104000729645E0E73DF40789F71092B2041092DA
:10105000B1041092B4041092B3041092B60410922A
:10106000B50450E040E06BE173E081EB94E0D4CC58
:10107000CF93DF93CDB7DEB72F970FB6F894DEBFCF
:101080000FBECDBF789484B5826084BD84B5816085
:1010900084BD85B5826085BD85B5816085BD809143
:1010A0006E00816080936E001092810080918100BB
:1010B00082608093810080918100816080938100B3
:1010C000809180008160809380008091B100846075
:1010D0008093B1008091B00081608093B0008091D6
:1010E0009100826080939100809191008160809353
:1010F0009100809190008160809390008091A10088
:1011000082608093A1008091A10081608093A10002
:101110008091A00081608093A00080912101826075
:101120008093210180912101816080932101809130
:10113000200181608093200180917A0084608093F7
:101140007A0080917A00826080937A0080917A00A0
:10115000816080937A0080917A00806880937A0021
:101160001092C100E0911B04F0911C0482E0808386
:10117000E0911704F09118041082E0911904F091A5
:101180001A0480E1808310922304E0911F04F091FF
:10119000200486E08083E0911D04F0911E0480818C
:1011A00080618083E0911D04F0911E04808188603D
:1011B0008083E0911D04F0911E048081806880830B
:1011C000E0911D04F0911E0480818F7D808382E375
:1011D00090E0A0E0B0E080930F0490931004A093FF
:1011E0001104B093120468EE73E080E090E0F1D94E
:1011F00069EAC62E64E0D62E8E010F5F1F4FD6011E
:101200008D916D011B861A861D861C861F861E8683
:1012100040E1B80190E060D2F80101900020E9F7C8
:101220003197AF01401B510BB801CE010A96F4DB98
:101230001A8219821C821B821E821D826091B10457
:101240007091B2046115710531F04091B50450916F
:10125000B604C801E1DB8E859F85AA84BB84ED803E
:10126000FE80E80EF91EA114B10409F439C0892BDF
:1012700079F0B701C801A8DB882391F129813A816F
:101280008D819E81B501820F931FA7D4FE82ED82CE
:1012900069817A816115710531F14D815E8181EB42
:1012A00094E0BADBC80189DBCE010A9686DBB1EB9C
:1012B000CB16B4E0DB0609F0A2CF0091B104109187
:1012C000B2040115110599F0F8018081882379F0A5
:1012D000082E000C990B70D4D8018D938D01F4CF9A
:1012E000C8015ADBD5CF81EB94E056DBDBCF88E237
:1012F00092E0D5D88EE692E0DADA86E292E0CFD8B4
:10130000D0DA84E292E0CBD884E092E0D0DA82E2D4
:1013100092E0C5D807D88FE192E0C1D847EBE42E20
:1013200044E0F42E04E112E05AE0A52EB12CF801BD
:10133000D0807181D701ED91FC910280F381E02D85
:1013400042E050E06D2DC7011995F701D186108656
:101350000190F081E02D0190F081E02DC7011995F9
:10136000882339F0D70118968C91189783601896C6
:101370008C935FD9F7016283738384839583B782EB
:10138000A6820C5F1F4FF2E1EF0EF11C47EDE41651
:1013900045E0F40661F60BEF13E037EDC32E35E0C0
:1013A000D32EC6011FDAD8016D937D938D939D9343
:1013B0008D01B0E1CB0ED11CE4E00B301E0789F7A4
:1013C00038D94B015C0180910A0290910B02A091E7
:1013D0000C02B0910D02AC01BD014854544F6F4F47
:1013E0007F4F84169506A606B70628F48816990638
:1013F000AA06BB0640F581E592E051D88EE692E060
:1014000056DA8FE492E04BD84CDA8DE492E047D87C
:1014100084E092E04CDA8BE492E041D80E949201A1
:1014200088E492E03CD880920A0290920B02A0924B
:101430000C02B0920D028092000290920102A092E2
:101440000202B09203029BEFC92E93E0D92E07ED62
:1014500015E02EE6222E22E0322E91E0F9E02F1642
:10146000F3E03F0609F090E0D8011C962D913C91E5
:10147000B3E02C313B0709F4C6C02752334009F4CE
:10148000C2C0D8011E962D913C9181E0B3E0223379
:101490003B0721F02D53334009F080E0992309F4F4
:1014A000B4C0882309F4B1C0C8019CD924E030E05D
:1014B00040E050E05CD129013A01F6018081918140
:1014C000A281B38184159505A605B7050CF0A4C0CB
:1014D000D8011E968D919C91EAD986E492E00E94F3
:1014E0004F028092000290920102A0920202B092FA
:1014F0000302D6014D925D926D927D926D01005F67
:101500001F4FB6E007311B0709F0A7CF84E1C82EB3
:1015100082E0D82E07EB14E0F80180858B7F80876E
:101520000190F081E02D0190F081E02DC801199526
:10153000782ED80118968C9186958170781609F4CA
:1015400078C077D8F801628373838483958380851C
:10155000F2E08F27D80118968C93F801808582FFDE
:101560001EC0D60112968D919C91A1D9F80190854B
:10157000892F847090FDA7C0882321F080E492E039
:101580000E944F0264E670E080E090E022D88092F2
:10159000000290920102A0920202B09203020E5E3B
:1015A0001F4FF4E0CF0ED11CE016F10609F0B4CFC6
:1015B00061E070E080E090E00CD8809100029091B2
:1015C0000102A0910202B0910302AC01BD014C598D
:1015D0005F4F6F4F7F4F84169506A606B70628F417
:1015E00088169906AA06BB0660F48AE392E00E9478
:1015F0004F028092000290920102A0920202B092E9
:1016000003029FD9DDCE81E049CFC801EBD822E0AB
:1016100030E040E050E04ECF481659066A067B069F
:101620000CF067CFF8018485958541D984E492E078
:1016300056CF0E941903F8012281338144815581DC
:101640001B012C01221A330A440A550AB201A101D6
:1016500086819781B0E0A0E0481759076A077B07A9
:1016600008F47BCF80858170781609F476CF0E94CC
:101670001903D80112966D937D938D939C931597C2
:1016800018968C91B1E08B278460F80180870E94C6
:101690001903D8011A964D905D906D907C901D971E
:1016A0006419750986099709F80166877787808B21
:1016B000918B0E941903D8011A966D937D938D9397
:1016C0009C931D974ACF882309F45CCF8CE392E06A
:1016D00057CF81EB94E071C9BB27FB015527AA279F
:1016E000880F991FAA1FA41710F0A41B83955051AF
:1016F000B9F7A05DAA3308F0A95DA193009779F727
:10170000B111B1931192CB0100C0DC01FC01672F34
:1017100071917723E1F7329704C07C916D937083C8
:101720006291AE17BF07C8F30895A1E21A2EAA1B53
:10173000BB1BFD010DC0AA1FBB1FEE1FFF1FA21781
:10174000B307E407F50720F0A21BB30BE40BF50B7E
:10175000661F771F881F991F1A9469F76095709507
:10176000809590959B01AC01BD01CF010895052E98
:1017700097FB16F400940FD057FD05D0D6DF07FC79
:1017800002D046F408C050954095309521953F4FC2
:101790004F4F5F4F089590958095709561957F4F5D
:1017A0008F4F9F4F0895EE0FFF1F881F8BBF07902D
:1017B000F691E02D19940F931F93CF93DF9382300E
:1017C000910510F482E090E0E0911906F0911A067C
:1017D00030E020E0B0E0A0E0309799F42115310529
:1017E00009F44AC0281B390B24303105D8F58A8109
:1017F0009B816115710589F1FB0193838283FE0151
:1018000011C0408151810281138148175907E0F0CE
:101810004817590799F4109761F012960C93129794
:1018200013961C933296CF01DF91CF911F910F91A8
:1018300008950093190610931A06F4CF2115310567
:1018400051F04217530738F0A901DB019A01BD019D
:10185000DF01F801C1CFEF01F9CF90931A06809311
:101860001906CDCFFE01E20FF31F81939193225011
:10187000310939832883D7CF209117063091180674
:10188000232B41F42091100230911102309318065D
:101890002093170620910E0230910F022115310579
:1018A00041F42DB73EB74091120250911302241B10
:1018B000350BE0911706F0911806E217F307A0F434
:1018C0002E1B3F0B2817390778F0AC014E5F5F4F96
:1018D0002417350748F04E0F5F1F509318064093AA
:1018E0001706819391939FCFF0E0E0E09CCFCF93D8
:1018F000DF930097E9F0FC01329713821282A091E6
:101900001906B0911A06ED0130E020E01097A1F41D
:1019100020813181820F931F209117063091180684
:101920002817390709F061C0F0931806E0931706ED
:10193000DF91CF910895EA01CE17DF07E8F54A81DC
:101940005B819E0141155105B1F7E901FB83EA83F3
:1019500049915991C40FD51FEC17FD0761F480819F
:1019600091810296840F951FE90199838883828172
:1019700093819B838A83F0E0E0E012968D919C91A5
:1019800013970097B9F52D913C911197CD010296CF
:10199000820F931F209117063091180628173907D8
:1019A00039F6309751F510921A0610921906B09335
:1019B0001806A0931706BCCFD383C2834081518100
:1019C000840F951FC817D90761F44E5F5F4F888158
:1019D0009981480F591F518340838A819B8193834A
:1019E00082832115310509F0B0CFF0931A06E093F8
:1019F00019069ECFFD01DC01C0CF13821282D7CF22
:101A00004F925F926F927F928F929F92AF92BF920E
:101A1000CF92DF92EF92FF920F931F93CF93DF93BA
:101A20008C01009791F4CB01DF91CF911F910F9121
:101A3000FF90EF90DF90CF90BF90AF909F908F90EE
:101A40007F906F905F904F90B6CEFC01E60FF71F2E
:101A50009C0122503109E217F30708F4AAC0D9010A
:101A6000CD91DC911197C617D70718F1C530D10574
:101A700070F0CE0104978617970748F0C61BD70B66
:101A80002297C193D1936D937C93CF0130DFC8012E
:101A9000DF91CF911F910F91FF90EF90DF90CF904A
:101AA000BF90AF909F908F907F906F905F904F907E
:101AB00008955B01AC1ABD0A4C018C0E9D1EA091CD
:101AC0001906B0911A06512C412CF12CE12C1097DB
:101AD00031F580911706909118068815990509F03F
:101AE0005CC04616570608F058C080910E029091CF
:101AF0000F02009741F48DB79EB7409112025091AA
:101B00001302841B950BE817F90708F052C0F093F5
:101B10001806E0931706F90171836083B8CF8D91A1
:101B20009C91119712966C90129713967C90139734
:101B3000A815B90559F56C0142E0C40ED11CCA14B0
:101B4000DB0420F1AC014A195B09DA011296159702
:101B500080F06282738251834083D9016D937C93BC
:101B6000E114F10471F0D7011396FC93EE931297F0
:101B70008ECF22968C0F9D1FF90191838083F301F4
:101B8000EFCFF0931A06E093190681CF4816590655
:101B900008F42C017D01D3019ACFCB010CDE7C012E
:101BA000009739F0AE01B8010FD0C801A0DE87015F
:101BB0006ECF10E000E06BCF9111089581568A51ED
:101BC00008F4805285580895FB01DC0102C00190A1
:101BD0000D9241505040D8F70895FB01DC0101906F
:101BE0000D920020E1F7089511E0C3E3D1E000E099
:101BF00005C0802FFE01D7DD2196011DC433D1071A
:0A1C000080E00807B1F7F894FFCF69
:101C0A00FFFFFFFF332E312E3900FFFFFFFF0000D9
:101C1A001B068000260048032700530321005E03A9
:101C2A002400660325006E032200760323007E0348
:101C3A00200087032900900328009C032B00A80397
:101C4A002A00B3032D00BC032C00C4033000CC03CC
:101C5A003100DC0300000000030265019B016902F8
:101C6A00CC01AA01BE010000000028032503526529
:101C7A00616C53696D476561722D474E5335333038
:101C8A0000454E435F464D535F4F555445525F449E
:101C9A004E00454E435F464D535F4F555445525F84
:101CAA00555000454E435F464D535F494E4E45528F
:101CBA005F444E00454E435F464D535F494E4E4585
:101CCA00525F555000454E435F434F4D5F494E4E5C
:101CDA0045525F444E00454E435F434F4D5F494E68
:101CEA004E45525F555000454E435F434F4D5F4F3F
:101CFA00555445525F444E00454E435F434F4D5F36
:101D0A004F555445525F5550005265616C53696D89
:101D1A00476561722D47464335303000454E435F73
:101D2A004844475F555000454E435F414C545F5508
:101D3A005000454E435F4844475F444E00454E437A
:101D4A005F414C545F444E0042544E5F4E41565FD1
:101D5A0046460042544E5F434F4D5F46460042544A
:101D6A004E5F4344490042544E5F4F42530042542F
:101D7A004E5F4D53470042544E5F46504C0042540A
:101D8A004E5F564E41560042544E5F50524F4300EA
:101D9A0042544E5F5A4F4F4D5F55500042544E5F6A
:101DAA005A4F4F4D5F444E0042544E5F444952458C
:101DBA0043540042544E5F4D454E550042544E5FC7
:101DCA00434C520042544E5F454E540042544E5FBB
:101DDA004E41565F434F4D5F544F470042544E5F4A
:041DEA00464D53000F
:00000001FF
